:020000040000FA
:020000000828CE
:020008000900ED
:10001000203084008001840A60300402031C0A2816
:100020002A16FF30C20041148316850185158312FC
:10003000850107309900C03083168100831231306A
:1000400090008E018F0100308B00003083168C00F1
:100050008312831631309B001C141A088312C500CA
:100060001D304502031C3528C50164000000C30B88
:100070004F28851940280A30C207031847284F28FF
:1000800041184F280A30C202031C4B284F28411048
:10009000FF30C2004F284114C20172214F288F083F
:1000A000031935288F01BF0100304502031D5D286B
:1000B0009821F42107222222352201304502031D16
:1000C00066289821F4210722A22235220230450217
:1000D000031D6F289821F42107222222EE220330EB
:1000E0004502031D78289821F4210722A222EE223E
:1000F00004304502031D8328BF163F179821F421C1
:1001000007222222352205304502031D8E28BF1604
:100110003F179821F4210722A222352206304502FA
:10012000031D9928BF163F179821F4210722222288
:10013000EE2207304502031DA428BF163F17982161
:10014000F4210722A222EE2208304502031DAE2828
:10015000BF163F179821F421BA22352209304502F3
:10016000031DB828BF163F179821F421BA22902208
:100170000A304502031DC2283F14BF163F179821BD
:10018000BA2235220B304502031DCC283F14BF167E
:100190003F179821BA2290220C304502031DD72820
:1001A0003F14BF163F1798210722222235220D3017
:1001B0004502031DE2283F14BF163F17982107226E
:1001C000A22235220E304502031DED283F14BF1632
:1001D0003F17982107222222EE220F304502031DED
:1001E000F8283F14BF163F1798210722A222EE22BB
:1001F00010304502031D03293F14BF14BF163F17DB
:1002000098210722352211304502031D0E293F1483
:10021000BF14BF163F1798210722902212304502C3
:10022000031D19293F14BF14BF163F179821072239
:10023000EE2213304502031D1E29D221143045023F
:10024000031D29293F14BF14BF163F17B3212222D3
:10025000352215304502031D33293F14BF14BF1644
:100260003F17B321AB2216304502031D3D29BF16AF
:100270009821F42107222222352217304502031D3E
:100280004729BF169821F4210722A22235221830CF
:100290004502031D5229BF163F179821F42107225A
:1002A0007E22902219304502031D5B2948225A22E2
:1002B0006C227E2290221A304502031D64294822B6
:1002C0005A226C22A22290221B304502031D6C2967
:1002D0003F171A23222235221C304502031D7129A3
:1002E00045233528C50A1D3045020318C501AA015A
:1002F0002A16AB01A801B001B101B201B301B401EA
:10030000B501B601B701B801B901BA018B134508AF
:1003100083161C159A0031309B0055309D00AA3081
:100320009D009C149C1892291C1183128B170800A5
:10033000B00A0A303002031C0800B11C8512B11843
:100340000512FA30311C2D303002031C0800B10AAE
:100350003F1CB1100130BF1EB100B11C8516B11891
:100360000516B0010800B00A0A303002031C08006C
:100370008512051205111E30B118643031198C3008
:100380003002031C08000310B10DB1193114B1087B
:100390000319311431188516B118051631190515D0
:1003A000B0010800B00A0A303002031C08008512B0
:1003B00005120511851005107D30311C53303002B7
:1003C000031C0800B10A0330B105B10803198516F2
:1003D00003190516B1180515B11885143118F2293D
:1003E000B1180514B0010800B20A0A303202031C29
:1003F00008000512FF30331C37303202031C08009E
:10040000B30A01303F1FB3000516B2010800B40A59
:100410000A303402031C0800B51C0511B5188510FC
:10042000F630351C32303402031C0800B50ABF1CFC
:10043000B51001303F1FB500B51C0515B518851462
:10044000B4010800B60A0A303602031C0800851001
:10045000F030381C1E303602031C0800B80A013088
:100460003F1FB8008514B6010800B90A0A303902E6
:10047000031C08000510F3303A1C28303902031C15
:100480000800BA0A01303F1FBA000514B90108007C
:10049000B00A1430311C46303002031C08008512AB
:1004A0006730311C73303002031C0800B10A851616
:1004B000B0010800B20A1430331C46303202031C6B
:1004C000080005126630331C72303202031C08002B
:1004D000B30A0516B2010800B40A1430351C4630C0
:1004E0003402031C080005116230351C6C303402E4
:1004F000031C0800B50A0515B4010800B60A14303B
:10050000381C46303602031C080085106730381C42
:1005100071303602031C0800B80A8514B6010800C1
:10052000B90A14303A1C46303902031C0800051081
:1005300064303A1C6E303902031C0800BA0A0514F4
:10054000B90108003608B60B08000508023A850014
:10055000C830B60008003608B60B0800B70A371CCA
:1005600008000508023A85000510851C0514A03016
:10057000B6000800A80FC32A1E30A8000310AA0D59
:10058000AA1AAA15AA122808AB000130AA19AB02B0
:1005900068302A050319CE2A851005152A132B0861
:1005A0000E020318D92A14302A050319D92A8514F2
:1005B00005118F08031D080064002B080E02031CA0
:1005C000D92A14302A050319E72A85100515283081
:1005D0002A050319ED2A851405110800A80FF72A2A
:1005E0001E30A8000310AA0DAA1AAA15AA122808DC
:1005F000AB000130AA19AB0268302A05031D0510B3
:100600002A132B080E020318092B14302A05031D88
:1006100005148F08031D080064002B080E02031C3C
:10062000092B14302A05031D051028302A05031D47
:1006300005140800B00A1E30B1193230311A1E30CC
:100640003002031C08008512051205110230311911
:100650002830B1196430311A96303002031C08007A
:100660000310B10DB11A3114B10803193114193046
:100670003105031D85161A303105031D05161C3082
:100680003105031D0515B0010800B00A1E30B11A6E
:100690003230311B1E303002031C08008512051257
:1006A0000511851005100230311A2830B11A643056
:1006B000311B96303002031C08000310B10DB11B32
:1006C0003114B1080319311461303105031D851649
:1006D00062303105031D051664303105031D051513
:1006E00068303105031D851470303105031D051474
:0406F000B00108004D
:084000000000010001000500B1
:02400E00CC01E3
:00000001FF
